:020000001028C6
:020008003F298E
:10002000B320BD20AB01AC01AD01AE013230A30065
:10003000A400A500A6004920602077208E2083160A
:1000400003308100831281018B01A520AB202008A1
:10005000A300AB202008A400AB202008A500AB2003
:100060002008A600AB202008A700AB202008A8008D
:10007000AB202008A900AB202008AA00AB202B3021
:10008000A302A402A502A6024920602077208E20A8
:10009000242823082B02AF0003195F2803185728D0
:1000A0000616000006100614AF0F50285D28061231
:1000B000000006100614AF0B57282308AB000800F9
:1000C00024082C02AF000319762803186E280616A0
:1000D000000086108614AF0F6728742806120000EF
:1000E00086108614AF0B6E282408AC000800250883
:1000F0002D02AF0003198D2803188528061600006D
:1001000006110615AF0F7E288B2806120000061177
:100110000615AF0B85282508AD00080026082E021D
:10012000AF000319A42803189C28061600008611A6
:100130008615AF0F9528A228061200008611861595
:10014000AF0B9C282608AE00080081018B01AB2074
:100150000B1DA6280800051EAB28051AAD280108AE
:10016000A000810108008501061486140615861575
:100170008316E0308600831208006430A100061266
:1001800006100614861086140611061586118615AB
:10019000A10BC02808006430A10006160610061442
:1001A000861086140611061586118615A10BCE2819
:1001B00008002730970010309600F8201A089B009E
:1001C00003309700E8309600F8201A089C000030B1
:1001D000970064309600F8201A089D0000309700C0
:1001E0000A309600F8201A089E0014089F000800A4
:1001F0009A019A039A0A0021031CFA281421080084
:10020000A201170898001608940203180A29980AF0
:100210000319221418089502031C10290310112930
:100220000314221803140800A201160894070318E7
:10023000950A0319221417089507221803140800B9
:100240008316051627308100831200308B000800CA
:100250008316273081008312080083162530810021
:100260008312080083162130810083120800A03019
:100270008B0095010800940000308B00080092006C
:10028000030E93000B19950A8B018B16130E830036
:06029000920E120E09009F
:00000001FF
